:1000000000308A00992900000A108A100A1182071C
:1000100028340C34013406340A108A100A1182077D
:1000200076347934733469346C3461346D3400342B
:100030002E308400000803192C280130A100A001F3
:10004000A00B2028A10B1F284A30A000A00B2628B7
:1000500000000000800B1D28003406080F39B50091
:10006000340EA000F030A0052008F03935048600D9
:100070000615831606110000831206118316061159
:1000800083120034B208031D4728861048288614BE
:10009000831686108312B30E3308B4002D20B30EDE
:1000A0003308B4002D200D30A000A00B55280034DB
:1000B0001430AE0018200F30831686058312861088
:1000C0008316861083120611831606118312AB0164
:1000D0002B08023C031C74280230AE0018200330A9
:1000E000B4002D20AB0A68280D30A000A00B7628A4
:1000F0000230B4002D200D30A000A00B7D28AB01F4
:100100002B08023C031C90282B080420AC00B201F1
:100110002C08B30042200230AE001820AB0A802821
:100120008A11DB2901302E02B0002F08023C031D8A
:100130009B284030B00730088038B100B201310848
:10014000B300422000342D08A0000C302002031917
:10015000B6280A3020020319BE280D3020020319E8
:10016000C428083020020319C928CE28B201013062
:10017000B30042200230AE001820DA280130AE0071
:100180000230AF009220DA280130AE00AF0092209A
:10019000DA28B2011030B3004220DA282D081F3CC3
:1001A000031CD4280730AD050130B2002D08B30080
:1001B0004220DA2800342E08A1012D020318E3287A
:1001C0002D08A000EF28A0010830AF00AD0DA00D54
:1001D0002E0820020318A000A10DAF0BE628003462
:1001E0002B08A000AB1BF8282C1D02292030FD286D
:1001F000A009A00A2008AB002D30A100AD00A3206B
:100200002C1DAC152B08AD006430AE00DB2020089F
:10021000AB0021083030031D14292C18AC15AC1983
:100220001A292C1A20301629AC112C12A1072108EA
:10023000AD00A3202B08AD000A30AE00DB20200863
:10024000AB0021083030031D2929AC192D292C1AA7
:100250002030A1072108AD00A3203030AB072B08C8
:10026000AD00A3200034AE012E08033C031C8B29F3
:100270002D08A0002E08A100031942290310A00C8C
:10028000A10B3E29003020180130013C031D6029DC
:10029000A91129088316870083128715A630A000AC
:1002A000A00B50290000A91129088316870083128A
:1002B0008711F930A000A00B5B29000000008929FC
:1002C000A911290883168700831287155330A000CF
:1002D000A00B6829A91129088316870083128711AA
:1002E000A630A000A00B72290000A91129088316CE
:1002F0008700831287155330A000A00B7D29A91118
:10030000290883168700831287115330A000A00BA1
:100310008729AE0A342900340F30AD0033212C0870
:10032000AD0033212B08AD0033212B08AD00332164
:10033000003484011F308305073083169F00FF308F
:100340008312A900AA01043083169F0083121F089C
:10035000383901389F009412A912290883168700A2
:10036000831229162908831687008312A9112908E8
:100370008316870000308312940083169400831242
:10038000A001A01DCB290730810181308400000825
:10039000C0390F3880006400813084000008C03903
:1003A0002004800090010030A100920000308316EC
:1003B0009200831258280C30AD00A3200730AE0005
:1003C0000230AF009220AB012B080C20AB0AAD002D
:1003D000A32007302B02031DE4290030A1001F08D1
:1003E000C73921049F000130AE00AF0092201F15D5
:1003F0001F19F8291E081E0EA7000F30A705583038
:10040000AD00A3203A30AD00A3202030AD00A320E2
:100410002708AB001830AC00F0200630AB002030CD
:10042000AD00A320AB0B0F2A0830A1001F08C7396D
:1004300021049F000130AE000230AF0092201F1552
:100440001F19202A1E081E0EA8000F30A8055930BB
:10045000AD00A3203A30AD00A3202030AD00A32092
:100460002808AB001830AC00F0200630AB0020307C
:10047000AD00A320AB0B372A291229088316870069
:10048000831207162913290883168700831207177A
:100490000130AE0018202912290883168700831224
:1004A00007122708AB00AC018C210A30AE001820DF
:1004B0002808AB000130AC008C21291329088316D1
:0A04C000870083120713ED29630083
:02400E00F13F80
:00000001FF
